:020000040000FA
:0400000068303A2802
:08000800A000030EA100831209
:1000100005191028831601178312B23081002B288E
:1000200083160113831203140B190310A80DA90DD5
:10003000AA0DAB0DAC0DAC16FF302C02031D2B2806
:10004000FA302B02031D2B2831152A08AF0029088E
:10005000AE002808AD008B100B11210E8300A00EFE
:04006000200E090065
:0C007400203084008001840A80300402E7
:10008000031C3C281230B0005A2183160C30850521
:1000900087018312850187010730990000309A009B
:1000A000103083168E008312603083168F00831207
:1000B0000030831691009F008312C83083168100A0
:1000C000831231309000003083168C008312103080
:1000D0008B00831600309B001C141A088312BC008E
:1000E000851D71213C1C7C28831610309B001C143C
:1000F0001A088312BD00662181018E018F010B1148
:100100008B100B108C018B179420311997203C21F8
:10011000B30B9228031085190314B90DF03039027E
:100120000319EF2097218428640032100800311150
:100130000130B7008B132030370783169B001C1447
:100140001A088312A4001030370783169B001C1472
:100150001A088312A300A6000230A6060030370753
:1001600083169B001C141A088312A200A7000130FA
:10017000A7068B17321CC22822090339A200A30943
:10018000A409A50924082F02031DE92823082E022B
:10019000031DD72822082D02031DE928013037024C
:1001A000031DD7283D18D7283D143E145B2126088F
:1001B0002E02031DE92827082D02031DE92801301E
:1001C0003702031DE8283D1CE8283D103E145E213F
:1001D000E928B70A02303702031808009A280130CC
:1001E000B600B300B400B500B70085018701B113B4
:1001F0009420B30B0B29031085190314B90DF030AB
:10020000390203193229B40B0B29013037020319C3
:1002100062219630B400311DF8283111321C1529A5
:100220002D090339AD00AE09AF092F1CF8288E0146
:100230008F010C1CF8280C102E1EF8288B13203070
:100240003707BB002F08BA00452110303707BB0025
:100250002E08BA00452100303707BB002D08BA0030
:1002600045218B1785018701B70AB6010230370295
:10027000031CF828662108003E1C08003E101030C0
:10028000BB003D08BA00452108008B133A088316CD
:100290001C159A0083123B0883169B0055309D0065
:1002A000AA309D009C1464009C1853291C118312D1
:1002B0008B17080008000130BD00080087010530D9
:1002C000D40008000508333A8500080001303D02DB
:1002D00003196B2908000130D40056150730D300EC
:1002E0000800B601B301B4013C1C7929BC01BC145F
:1002F0007B29BC013C143C08B60064007F2980299E
:100300008129822983293330B41B8500B41F8501DC
:10031000B30B7D29B40B7D290310B60CB608031D61
:100320007D290030BB003C08BA00452108008F0839
:10033000031908008E018F01D0080319E729D00F97
:10034000B42956180516D618851656190514D61947
:100350008514D60158180512D81885125819051099
:10036000D8198510D801E7295008D100561805166C
:10037000D618851656190514D619851451080E027B
:100380000318CE2958180512D818851258190510C7
:10039000D8198510FF305002031908008F08031D7B
:1003A0000800942051080E02031CCE29561805128D
:1003B000D618851256190510D61985105818051625
:1003C000D818851658190514D81985140800003056
:1003D0005302031D002A3D18F829051A581401304C
:1003E000051AD000851AD8140130851AD0000800EB
:1003F0000130D40056140130D0000130D300080081
:10040000051A062A5614851AD814082AD614581420
:100410000130D000D40B080001305302031D1A2A0A
:10042000D6150530D4000230D3003D180800D6019F
:10043000D301080002305302031D2C2A56158714DD
:10044000D8150330D4000330D3003D1808008701CD
:10045000D601D301D815080003305302031D3C2AEE
:10046000871407150330D4000430D3003D1808006A
:100470008701D3015815080004305302031D4D2A8B
:100480008714071507140330D4000530D3003D1836
:1004900008008701D3015815080005305302031DD9
:1004A0005F2A87140715071487160330D400063017
:1004B000D3003D1808008701D30158150800063005
:1004C0005302031D722A871407150714871607168F
:1004D0000330D4000730D3003D1808008701D30152
:1004E0005815080007305302031D862A8714071584
:1004F00007148716071687150130D4000730D3007C
:100500003D1808008701D301581508000030D300BA
:020510000800E1
:084000000700030004000800A2
:02400E00CC33B1
:10420000010078007A007C007E007B0079007F004E
:104210007D007A0078007E007C00FF00FF00FF0038
:104220000000F200F600FA00FE00F200F600FA00CC
:10423000FE00F200F600FA00FE00FF00FF00FF00A3
:10424000010005000500050005000900090009003E
:1042500009000D000D000D000D00FF00FF00FF0024
:10426000FF00FF00FF00FF00FF00FF00FF00FF0056
:10427000FF00FF00FF00FF00FF00FF00FF00FF0046
:10428000FF00FF00FF00FF00FF00FF00FF00FF0036
:10429000FF00FF00FF00FF00FF00FF00FF00FF0026
:1042A000FF00FF00FF00FF00FF00FF00FF00FF0016
:1042B000FF00FF00FF00FF00FF00FF00FF00FF0006
:1042C000FF00FF00FF00FF00FF00FF00FF00FF00F6
:1042D000FF00FF00FF00FF00FF00FF00FF00FF00E6
:1042E000FF00FF00FF00FF00FF00FF00FF00FF00D6
:1042F000FF00FF00FF00FF00FF00FF00FF00DD00E8
:00000001FF
